:10000000020006020056787FE4F6D8FD75812802CA
:0200100009AB3A
:0D0013000200798F99752501E52570FC220A
:10002300020B67750840750901750D00750CC275E3
:100033000B01750A00750F017B007A0079087F01B7
:0F00430012083F7D017F01020B1AAE0702001663
:0700530002007D751C013263
:10005B00020C96EFD3940174809480500EEFC4334E
:10006B003354C0FFE58F54BF4FF58FE4FF22751C4F
:06007B000232751C033285
:10008300020C9AE517240BF8E605172278083007C7
:1000930002780BE475F0011208090206592000EBFF
:1000A3007F2ED2008018EF540F2490D43440D4FF15
:1000B30030040BEF24BFB41A0050032461FFE5188A
:1000C30060021518051BE51B7002051A30070D7831
:1000D30008E475F001120809EF0207C102004D742C
:1000E30003D2078003E4C207F5178B088A09890A3C
:1000F300E4F518F51AF51BE51860077F201200C117
:1001030080F57519FFC201C200C202C203C205C253
:1001130006C20812008FFF700D3007057F00120022
:10012300D2AF1BAE1A22B4255FC2D5C20412008F10
:10013300FF24D0B40A00501A75F00A781830D50598
:1001430008B6FF0106C6A426F620D5047002D20322
:1001530080D924CFB41A00EF5004C2E5D2040202BE
:10016300D2D20180C6D20080C0D20280BCD2D58058
:10017300BAD20580B47F201200C12002077401B5F2
:10018300180040F1120086FF1200C10200FAD208E3
:10019300D2068095120086FB120086FA120086F9B9
:1001A3004A4B700679A37A037BFF20022EE5186081
:1001B3002A7E008E8275830012067260060EEE653B
:1001C3001970F0C2D5EBC0E0EAC0E0E9C0E0EE127E
:1001D3000319D0E0F9D0E0FAD0E0FB120659FF6032
:1001E300AAEBC0E0EAC0E0E9C0E01200C1D0E0241D
:1001F30001F9D0E03400FAD0E0FBE5190460DCD566
:1002030019D980877BFF7A037915D202809C7910F4
:1002130080027908C206C2088008D2D5790A800410
:10022300790AC2D5E519047002F519E4FAFDFEFF57
:10023300120086FC7B08200113120086FD7B103020
:10024300000A120086FE120086FF7B20EC3382D563
:1002530092D55013C3E43000069FFFE49EFEE420D2
:1002630001039DFDE49CFCE4CBF8C201EC700CCFD0
:10027300CECDCCE824F8F870F38017C3EF33FFEE4C
:1002830033FEED33FDEC33FCEB33FB994002FB0F04
:10029300D8E9EB300105F8D0E0C448B201C0E00A68
:1002A300EC4D4E4F78207B0070C2EAB5190040BC7C
:1002B300C0E012031BD0F0D0E0200104C4C0E0C4AE
:1002C300B201C0F01200AAD0F0D5F0EB0200FA128E
:1002D300081901975302115801684C016442021531
:1002E3004F021D44021D49017D4302235502074667
:1002F30002074502074703C350016C2D01702E010D
:10030300932B01742301912003AC2A012C48000094
:10031300018B3F3F3F00790AA2D520031430050922
:10032300B910020404B9080104A2D5200602500141
:10033300042002689202B518005034C0E07F2030D8
:1003430003197F30A20272067205500F120372C2A4
:1003530002C206C205C2087F30800F300503E9C020
:10036300E01200C1300503D0E0F9D0E0B518CC307D
:1003730005177F30B9100C1200C17F583004077F76
:10038300788003B908031200C13002057F2D0200F3
:10039300C17F202008F87F2B2006F322920280CF12
:1003A300286E756C6C2900D2011200863001F8C2E8
:1003B30001781830D50108F602012C2D5043495815
:1003C3001200862403B405004001E49003BE931297
:1003D30000B2743A1200B2D203751804020211EF8C
:1003E300D394077480948040037FFF22120659FE42
:1003F300D394037480948040037FFF22EF7044EE14
:10040300700B900001120672F45293529412065923
:100413006401700B9000011206724293F45294121D
:100423000659FE6402700A9000011206724293425A
:1004330094EE6403700D900001120672FEF4529361
:10044300EE4294EF64017046120659FE700B900061
:1004530001120672F452915292EE6401700B9000F5
:10046300011206724291F452921206596402700A02
:10047300900001120672429142921206596403706F
:100483000D900001120672FEF45291EE4292EF6457
:10049300027046120659FE700B900001120672F4A8
:1004A30052955296EE6401700B900001120672424F
:1004B30095F452961206596402700A9000011206CE
:1004C30072429542961206596403700D9000011210
:1004D3000672FEF45295EE4296EF640370461206DE
:1004E30059FE700B900001120672F452B152B2EE33
:1004F3006401700B90000112067242B1F452B21201
:1005030006596402700A90000112067242B142B2A7
:100513001206596403700D900001120672FEF45224
:10052300B1EE42B2EF64047046120659FE700B90AE
:100533000001120672F452B352B4EE6401700B90D0
:10054300000112067242B3F452B4120659640270E7
:100553000A90000112067242B342B41206596403B0
:10056300700D900001120672FEF452B3EE42B4EF26
:1005730064057046120659FE700B90000112067254
:10058300F452C952CAEE6401700B90000112067254
:1005930042C9F452CA1206596402700A9000011249
:1005A300067242C942CA1206596403700D900001D3
:1005B300120672FEF452C9EE42CAEF640670461286
:1005C3000659FE700B900001120672F452CB52CC06
:1005D300EE6401700B90000112067242CBF452CC10
:1005E3001206596402700A90000112067242CB424D
:1005F300CC1206596403700D900001120672FEF4CA
:1006030052CBEE42CCEF64077049120659FF7E00CD
:10061300700B900001120672F452E152E2EF640192
:100623004E700B90000112067242E1F452E2120680
:10063300596402700A90000112067242E142E2120A
:1006430006596403700D900001120672FFF452E123
:10065300EF42E27F0022BB010689828A83E02250B7
:1006630002E722BBFE02E32289828A83E49322BB50
:10067300010CE58229F582E5833AF583E0225006F1
:10068300E92582F8E622BBFE06E92582F8E222E5A7
:100693008229F582E5833AF583E4932275F00875A0
:1006A3008200EF2FFFEE33FECD33CDCC33CCC582AA
:1006B30033C5829BED9AEC99E58298400CF582EE66
:1006C3009BFEED9AFDEC99FC0FD5F0D6E4CEFBE44E
:1006D300CDFAE4CCF9A88222B800C1B90059BA0016
:1006E3002DEC8BF084CFCECDFCE5F0CBF97818EF71
:1006F3002FFFEE33FEED33FDEC33FCEB33FB10D772
:1007030003994004EB99FB0FD8E5E4F9FA22781832
:10071300EF2FFFEE33FEED33FDEC33FCC933C9108D
:10072300D7059BE99A4007EC9BFCE99AF90FD8E0BF
:10073300E4C9FAE4CCFB2275F010EF2FFFEE33FE91
:10074300ED33FDCC33CCC833C810D7079BEC9AE804
:1007530099400AED9BFDEC9AFCE899F80FD5F0DA85
:10076300E4CDFBE4CCFAE4C8F922EB9FF5F0EA9E72
:1007730042F0E99D42F0E89C45F022E8600FECC3AB
:1007830013FCED13FDEE13FEEF13FFD8F122BB01B3
:100793000DE58229F582E5833AF5830207E05007E8
:1007A300E92582F80207D3BBFE07E92582F8020791
:1007B300ECE58229F582E5833AF5830207F9BB016B
:1007C3000689828A83F0225002F722BBFE01F322BC
:1007D300E6FB08E6F908E6FA08E6CBF822E0F8A318
:1007E300E0F9A3E0FAA3E0FB22E2FB08E2F908E266
:1007F300FA08E2CBF822E493F8740193F9740293B4
:10080300FA740393FB22FAE6FB0808E6F925F0F6EF
:1008130018E6CA3AF622D083D082F8E493701274B1
:100823000193700DA3A393F8740193F5828883E475
:10083300737402936860EFA3A3A380DF8B118A1202
:100843008913EF640160030209A8752201F523F5FA
:1008530024F525F526F527F528FFEFC3948074804A
:100863009480500F74802FF582E43400F583E4F014
:100873000F80E7E4FFEFC3948074809480500F747B
:10088300002FF582E43400F583E4F00F80E7AB1129
:10089300AA12A913120659FFE598543F4FF598EF92
:1008A30064C06008EF6440600302095790000212BD
:1008B30007917F007E607D547C001206DB8F178ECC
:1008C300168D158C14E4FFFE7D01FCAB17AA16A947
:1008D30015A814C312076D40037FFF22C3E49517C5
:1008E300F517E49516F51674019515F515E49514A9
:1008F300F514AB11AA12A913900001120672640237
:100903007026538EEF438E01538EF7438E04AF1739
:10091300AE16AD15AC14780812077E8FD68517D79F
:1009230053AFFB438E108066C28E538EFE5389BF36
:100933005389CF438E40AF17AE16AD15AC1478086C
:1009430012077E8F8D85178BC2AB5389BF538FFDE3
:10095300D28E803AAB11AA12A913120659FF7E0058
:10096300701490000812067264017005438E208093
:100973001D538EDF8018EF64804E701290000812B2
:10098300067264017005438780800353877FAB1130
:10099300AA12A9139000071206727004C29C800267
:1009A300D29C7F00227FFF22120C86120026D2AF38
:1009B3007BFF7A0C799E1200E830B2FD30B3FD3034
:1009C300B6FD30B7FD30B0FD7F0A7E00120C5C30FF
:1009D300B2FD30B3FD30B6FD30B7FD30B0FD7F0A58
:1009E3007E00120C5C120BB2E4F51C43870200007C
:1009F3000000000000E51C640170097BFF7A0C799C
:100A0300C21200E8E51C640270097BFF7A0C79D3FB
:100A13001200E8E51C640370097BFF7A0C79E41289
:100A230000E8E51C640470097BFF7A0C79F5120079
:100A3300E8E51C640570097BFF7A0D79061200E86E
:100A4300E4F51C051DE51D75F064842430FF1200D8
:100A530016E51D75F06484E5F075F00A842430FF13
:100A6300120016E51D75F00A84E5F02430FF12002C
:100A7300167BFF7A0D7917120C730209BCEFFBD3B7
:100A83009401748094805009EB7004C2A88002D250
:100A9300A8EDFF7E00D39403748094805029EF70F7
:100AA3000553B7FEC2B8EF64014E700553B7FED2CB
:100AB300B8EF64024E700543B701C2B8EF64034E4A
:100AC300700543B701D2B87F0022EFFBD3940174C2
:100AD3008094805009EB7004C2AA8002D2AAEDFF71
:100AE3007E00D39403748094805029EF700553B72C
:100AF300FBC2BAEF64014E700553B7FBD2BAEF6481
:100B0300024E700543B704C2BAEF64034E70054347
:100B1300B704D2BA7F0022EFFBD394017480948090
:100B23005009EB7004C2AC8002D2ACEDFF7E00D35F
:100B33009403748094805029EF700553B7EFC2BCBF
:100B4300EF64014E700553B7EFD2BCEF64024E70F1
:100B53000543B710C2BCEF64034E700543B710D210
:100B6300BC7F0022C0E0C083C082C0D075D000C06B
:100B730007309828C298E5287022C3E5269480742C
:100B83008094804003752600AF26052674002FF558
:100B930082E43400F583E599F0752705309905C2A1
:100BA30099752500D007D0D0D082D083D0E032759C
:100BB30008017B007A007908E4FF120BF1E4FD7F62
:100BC30001120A807508017B007A0079087F0112FF
:100BD3000BF1E4FD7F01120ACDE4FD7F01120C430A
:100BE300E4FD7F01120C29E4FD7F0102005EEFD3D7
:100BF30094017480948040037FFF22EF7010C289B8
:100C03001206597004C2888002D2887F0022EF64E2
:100C1300017010C28B1206597004C28A8002D28AF4
:100C23007F00227FFF22EFD3940174809480500DC4
:100C3300EFC43354E0FFE58F54DF4FF58FE4FF2219
:100C4300EFD3940174809480500CEFC454F0FFE50B
:100C53008F54EF4FF58FE4FF227DA37C08ED1D70C9
:100C6300011C144C70F7EF1F70011E144E70EA2222
:100C7300120659FF600C120016740129F9E43AFABE
:100C830080EE227509FFE4F508FB7A0079087F03FB
:100C93000203E2751C0432751C0532535443382099
:100CA3004558494E542057616B65757020546573E0
:100CB300742050726F6772616D6D65210D0A00CDEE
:100CC300E2D6D0B6CF494E5430BBBDD0D1202000A0
:100CD300CDE2D6D0B6CF494E5431BBBDD0D12020C2
:100CE30000CDE2D6D0B6CF494E5432BBBDD0D120D1
:100CF3002000CDE2D6D0B6CF494E5433BBBDD0D1C0
:100D0300202000CDE2D6D0B6CF494E5434BBBDD05F
:0D0D1300D1202000B4CEBBBDD0D10D0A0010
:00000001FF
